:020000040000FA
:060000008A110A12052816
:10000800090074221B226122831603130716871521
:100018000C3083120313A100A521DD30F20001305A
:10002800F3008A30F7000330F8006723DD30B000B2
:100038000130B1003C230130F4009D217A210330C6
:10004800F4009D21DD30F2000130F3009A30F70012
:100058000330F8006723DD30B0000130B1003C23E5
:100068000130A800A6012423DD30F2000130F3009E
:10007800A530F7000330F8006723DD30B000013009
:10008800B1003C230330F4009D217A21A801A60188
:100098002423DD30F2000130F300B030F7000330E4
:1000A800F8006723DD30B0000130B1003C23013097
:1000B800A800A60124230A30A70091220330F400E7
:1000C8009D217A210D30A7009122A801A6012423A1
:1000D800DD30F2000130F300BA30F7000330F800E9
:1000E8006723DD30B0000130B1003C230330F40059
:1000F8009D217A21A801A6012423DD30F2000130D8
:10010800F300C530F7000330F8006723DD30B00096
:100118000130B1003C230130A800A6012423093096
:10012800A70091220330F4009D217A21A801A6019D
:100138002423DD30F2000130F300CE30F700033025
:10014800F8006723DD30B0000130B1003C230E30E9
:10015800A70091220330F4009D21A801A6012423C1
:10016800DD30F2000130F300D830F7000330F8003A
:100178006723DD30B0000130B1003C230130A80016
:10018800A60124230A30A70091220930A700912252
:100198000330F4009D21A801A6012423DD30F200DC
:1001A8000130F300E830F7000330F8006723DD3052
:1001B800B0000130B1003C230130A800A60124237F
:1001C8000D30A70091220E30A70091220330F400D1
:1001D8009D217A21A8010430A6002423DD30F200F5
:1001E8000130F300F930F7000330F8006723DD3001
:1001F800B0000130B1003C230130A8000430A60053
:100208002423DD30F2000130F3000230F70004301F
:10021800F8006723DD30B0000130B1003C23F43032
:10022800F2000130F3008F210A30B3000B30A70031
:100238009122F430F2000130F3008F210C30A70036
:100248009122F430F2000130F3008F21B30B1A2908
:100258007A21A801A6012423DD30F2000130F30041
:100268000A30F7000430F8006723DD30B0000130B1
:10027800B1003C230130A800A6012423DD30F200A0
:100288000130F3001B30F7000430F8006723DD303D
:10029800B0000130B1003C230230F4009D210B3046
:1002A800A7009122A90186220530F4009D21013082
:1002B800A90086227A21A801A60124230C30A700D0
:1002C8009122DD30F2000130F3002530F7000430D0
:1002D800F8006723DD30B0000130B1003C23033063
:1002E800F4009D212228782963007829AF10013075
:1002F800A500D5220430F200F3018F218030A5003B
:10030800D5220C30F50088290C30F000F00B8A2932
:10031800F50B88290800F30A6C30F1000B30F00067
:10032800F00B9429F10B9229F20B9029F30B9029E9
:100338000800E830F2000330F3008F21F40B9D2908
:1003480008008316031394178312031314169413C7
:100358000C302102031DB82994151411941014109F
:10036800273083160313930083120313A108031D78
:10037800C129941114159414141003302102031D7B
:10038800C92994111415941414149416080094137C
:10039800230893000C2283160313111FD829FF305A
:1003A80083120313A000DB2983120313A001941FF7
:1003B800E12921080A3C0318CB2921080A3C031823
:1003C8001416080021080A3C0318F12983160313A0
:1003D8001114831203130C22F52983160313941D99
:1003E800F12983120313080021080A3C0318052A7F
:1003F800831603131419FC291115831203130C22F5
:10040800092A83160313141E052A831203130800EE
:10041800A201A20AFF30220203181A2A8C1D0D2AF3
:100428008C1108008C1D0D2A8C1108000800A101F0
:1004380008000F30F200F3018F210330A500D52208
:100448000530F200F3018F210330A500D5220130D9
:10045800F200F3018F210330A500D5220130F2000C
:10046800F3018F210330A500D5220130F200F301FA
:100478008F210230A500D5220130F200F3018F212F
:100488002830A500D5220130F200F3018F210C306D
:10049800A500D5220130F200F3018F210130A5001B
:1004A800D5220F30F200F3018F210630A500D522A6
:1004B8000130F200F3018F217A290C30A100A52127
:1004C8000130AA000230F200F3018F210230B4009B
:1004D8004E30AB001D22B40B6C2A0C30AC00080067
:1004E800831603139F13831203131F10831603131A
:1004F8009F111F159F141F10831203138501860176
:1005080087010800A9080319AA012903031D8E2AD7
:100518000130AA00AF10A501D52AAF102703031D8B
:10052800982A0C302C04A9000C302702031D9F2A9E
:100538000C302C04A900A708031DA52A0B302C0594
:10054800A9000B302702031DAC2A0B302C05A9008B
:100558000A302702031DB32A0A302C04A9000D30E3
:100568002702031DBA2A0D302C05A90009302702DD
:10057800031DC12A09302C04A90009302702031DD4
:10058800C82A09302C04A9000E302702031DCF2ADF
:100598000E302C05A9002908A500D5222908AC0091
:1005A8000800AF1CD92A2414DA2A2410A410A41194
:1005B8002A18A415E6212B08A300CB21A413A51BF8
:1005C800A4172413251B2417A412A51AA416241251
:1005D800251A241624112408A300CB212415240845
:1005E800A300CB2124112408A300CB21A413A5190F
:1005F800A417241325192417A412A518A416241225
:100608002518241624112408A300CB212415240816
:10061800A300CB2124112408A300CB21F8210C30FE
:10062800AC000D30F000F00B172B1030250203182A
:10063800232B2508073C0318232B2508AC000800AA
:10064800AF102808013C03182D2B0230A8021430E3
:10065800A6072808F5004030F9005B232608700734
:10066800B50080303504A500D5220530F50088296D
:10067800300884008313311883170008AD00AD08D3
:1006880003190800AF14B20101302D02031C5A2BC4
:10069800B20A320830078400831331188317000820
:1006A800A500D5222D083202031C4C2B0800F001AE
:1006B80075087918F0070310F90C0310F50DF908FF
:1006C800031D5C2B080072088400831373188317BA
:1006D8008323F5008000F2077A2B720884008313C5
:1006E800731883178323F500F607F207F508031933
:1006F80008008323840A8000F50B7D2B0800780806
:100708008A007708F70A0319F80A82000F34473479
:100718007234653461347434203443346F3477343C
:100728002034423461347334693463340A345334C2
:1007380054344134523454342034543445345334CA
:1007480054340A3444344934533450344C344134E6
:10075800593420344F344E340934433475347234A8
:1007680073346F34723420344F344E340A34433483
:100778007534723473346F34723420344F344634E1
:100788004634083446344C344134533448342034E5
:100798004F344E34093446344C344134533448349D
:1007A80020344F34463446340F34433455345234AD
:1007B8005334523420342634203446344C345334A1
:1007C800483420344F344E34103443345534523482
:1007D8005334523420342634203446344C34533481
:1007E800483420344F3446344634083446346C3464
:1007F80061347334683469346E346734073444348C
:100808006934733470346C3461347934103444345A
:100818004934533450344C34413459342034263418
:1008280020344234413443344B344C342E3409346C
:1008380046344F345234203435342034533445341C
:100848004334083445344E34443420345434453425
:04085800533454348D
:02400E007A3FF7
:00000001FF
